:020000040000FA
:02000000062ACE
:08000800A300030EA200C503D2
:1000100003190B2834281330C5003A205420A5209A
:100020002F1C1828A703031D18286430A700A8094F
:100030000721A403FF302402031D34280930A40043
:10004000A503FF302502031D34280930A500A603AF
:10005000FF302602031D34280330A4000130A50020
:100060000530A6003018CE200B11220E8300A30EFF
:10007000230E09002B1808002D18080029184928FC
:100080000618080031102F143010FA30AA00291475
:100090000800AA03031D08002910A10A0630210246
:1000A000031D0800A1010800291808002D180800E8
:1000B0002B1863288618080031102F143010963042
:1000C000AC002B140800AC03031D08002B100030FB
:1000D0002102031D7228B20A0A303202031D0800F1
:1000E000B201080001302102031D7D28B30A0A3045
:1000F0003302031D0800B301080002302102031D72
:100100008828B40A06303402031D0800B401080030
:1001100003302102031D9328B50A0A303502031D5E
:100120000800B501080004302102031D9E28B60A0C
:1001300006303602031D0800B6010800B70A0A306F
:100140003702031D0800B70108002B180800291802
:1001500008002D18C928861B08002F1CC228FA3059
:10016000AE002D1431102F1030143208B8003308AF
:10017000B9003408BA003508BB003608BC0037089F
:10018000BD000800FA30AE002D1431142F103010CD
:100190000800AE03031D08002D100800BD03FF304A
:1001A0003D02031DFA280930BD00BC03FF303C02AC
:1001B000031DFA280530BC00BB03FF303B02031DC2
:1001C000FA280930BB00BA03FF303A02031DFA28AF
:1001D0000530BA00B903FF303902031DFA2809308F
:1001E000B900B803FF303802031DFA2831102F1070
:1001F000301008003808B2003908B3003A08B400DB
:100200003B08B5003C08B6003D08B7000800311CAB
:100210001029BE01BF01C001C101C201C3015A2999
:100220002F1C4B29281C3E2900302102031D1B29AD
:100230000F30BE005A2901302102031D22290F3040
:10024000BF005A2902302102031D29290F30C000A6
:100250005A2903302102031D30290F30C1005A29C9
:1002600004302102031D37290F30C2005A290530FE
:100270002102031D5A290F30C3005A293208BE003B
:100280003308BF003408C0003508C1003608C2007A
:100290003708C3005A29301C5A293808BE003908CB
:1002A000BF003A08C0003B08C1003C08C2003D083E
:1002B000C3005A29A003FF302002031D6129053025
:1002C000A00000302002031D6C291F308500833000
:1002D00086003E08C400A32901302002031D7729AF
:1002E000C33086001E3085003F08C400A3290230B9
:1002F0002002031D8229C33086001D30850040087E
:10030000C400A32903302002031D8D29C3308600B9
:100310001B3085004108C400A32904302002031DBE
:100320009829C3308600173085004208C400A329ED
:1003300005302002031DA329C33086000F3085003D
:100340004308C400A32900304402031DAC29061150
:10035000861106128612080001304402031DB529D9
:100360000615861106128612080002304402031D8B
:10037000BE290611861506128612080003304402B3
:10038000031DC729061586150612861208000430BB
:100390004402031DD0290611861106168612080094
:1003A00005304402031DD92906158611061686124A
:1003B000080006304402031DE229061186150616C0
:1003C0008612080007304402031DEB290615861526
:1003D00006168612080008304402031DF42906118F
:1003E000861106128616080009304402031DFD29F5
:1003F000061586110612861608000F304402031DEA
:1004000008000615861506168616080083120313C3
:100410008501860107309F00831603130030810099
:10042000003085008330860083120313203084005F
:100430008001840A80300402031D182A0330A400BE
:100440000130A5000530A6001330C5000430A1001E
:10045000FA30AA009630AC00FA30AE006430A70043
:0C04600031148101A0308B00352A352AB0
:02400E00223F4F
:104200002800430029004600610062007200690036
:10421000630065002000530069006E0063006500C4
:10422000720065002000300032002F0030003300A3
:0A4230002F0032003000300037008C
:00000001FF
